:100000000C94CC020C9404030C9404030C9404038D
:100010000C9404030C9404030C9404030C94040344
:100020000C9404030C9404030C945A260C942C276F
:100030000C9439210C9404030C9404030C940403D1
:100040000C9404030C9404030C9404030C94040314
:100050000C9404030C94C1210C9404030C94040329
:100060000C9404030C9404030C9404030C940403F4
:100070000C9404030C9404030C9404030C940403E4
:100080000C9404030C9404030C9404030C940403D4
:100090000C9404030C9404030C9404030C940403C4
:1000A0000C9404030C9404030C940403CC05CC05B9
:1000B000F805F80560067E0696079607890622076A
:1000C000330733079927C027B828C027B8280C283A
:1000D0002F28B8288628952829001E001F002000F8
:1000E00021002200230024002500260027002D00E7
:1000F0002E002A0035002B0014001A0008001500FD
:1001000017001C0018000C00120013002F00300014
:1001100031004B0039000000040016000700090000
:100120000A000B000D000E000F0033003400280001
:100130004E000000E1001D001B0006001900050034
:1001400011001000360037003800E50052004C0066
:10015000E000E3000000E200000000002C000000CE
:100160000000E6000151E400500051004F00010082
:100170003A003B003C003D003E003F004000410093
:10018000420043004400450001004A000100010014
:100190000100010001000100010001000100010057
:1001A00046004700480001004D0001000000C35C0C
:1001B000CE5CCF5CD05CD15CD25CD35CD45CD55CD3
:1001C000D65C01000100490000000100C45CC65C6F
:1001D000C75CC85CC95CCA5CCB5C01000100010063
:1001E000010001000100005C0100000001000000AE
:1001F00000000100000000000100010001000100FA
:100200000100010000047F3F1F643214643214783F
:100210003C1E1E140A052223252628292A2C2D2FB0
:100220003032333536383A3B3D3E4042434547490C
:100230004A4C4E5051535557595A5C5E6062646641
:1002400068696B6D6F71737577797B7D7F8183854D
:1002500087898A8C8E90929496989A9C9E9FA1A34F
:10026000A5A7A8AAACAEAFB1B3B4B6B8B9BBBCBE73
:10027000BFC1C2C3C5C6C7C9CACBCCCDCED0D1D2EF
:10028000D2D3D4D5D6D7D7D8D9D9DADADBDBDBDCF1
:10029000DCDCDCDCDDDDDDDDDCDCDCDCDCDBDBDB9D
:1002A000DADAD9D9D8D7D7D6D5D4D3D2D2D1D0CEFD
:1002B000CDCCCBCAC9C7C6C5C3C2C1BFBEBCBBB902
:1002C000B8B6B4B3B1AFAEACAAA8A7A5A3A19F9E80
:1002D0009C9A98969492908E8C8A89878583817F48
:1002E0007D7B79777573716F6D6B69686664626029
:1002F0005E5C5A5957555351504E4C4A49474543F5
:1003000042403E3D3B3A3836353332302F2D2C2A91
:10031000292826252322FFAA7F554000010101013B
:1003200001010101010202020202020202020303B0
:100330000303030303030404040404040405050580
:100340000505060606060607070707070808080842
:10035000090909090A0A0A0B0B0B0C0C0C0D0D0DEF
:100360000E0E0E0F0F0F1010111111121213131485
:1003700014151516161717181819191A1A1B1B1CFD
:100380001D1D1E1E1F202021222223242425262657
:10039000272829292A2B2C2D2D2E2F30313232338C
:1003A0003435363738393A3B3C3D3E3F4041424395
:1003B0004445464748494A4C4D4E4F505153545579
:1003C0005658595A5B5D5E5F616264656668696B29
:1003D0006C6D6F7072737577787A7B7D7E808283A7
:1003E0008587888A8C8E8F91939596989A9C9EA0EB
:1003F000A2A3A5A7A9ABADAFB1B3B5B7BABCBEC0F8
:10040000C2C4C6C9CBCDCFD1D4D6D8DBDDDFE2E4C0
:10041000E7E9EBEEF0F3F5F8FAFDFF240343007291
:100420000061007A00790020004B006500790062CD
:10043000006F006100720064002000360038000088
:10044000000E036300680065006E00740037000052
:10045000000403090409023B00020100A0FA090498
:1004600000000103010100092111010001224000E7
:1004700007058103080001090401000103000000D1
:1004800009211101000122B60007058203200001A5
:100490001201000200000008EDFEDE13010001025F
:1004A000000105010902A10185020901A100050958
:1004B000190129081500250195087501810205011A
:1004C000093009311581257F9502750881060938A3
:1004D0001581257F950175088106050C0A380215DE
:1004E00081257F950175088106C0C005010980A19D
:1004F00001850319012AB700150126B7009501757A
:10050000108100C0050C0901A101850419012AA070
:1005100002150126A002950175108100C005010990
:1005200006A1018506050719E029E71500250195B3
:1005300008750181020507190029EF1500250195AD
:10054000F0750181020508190129059505750191CC
:1005500002950175039101C005010906A101050776
:1005600019E029E71500250195087501810295011B
:10057000750881010507190029FF150026FF009560
:100580000675088100050819012905950575019171
:1005900002950175039101C011241FBECFEFDAE06F
:1005A000DEBFCDBF04B603FE18C080910C0490914D
:1005B0000D04A0910E04B0910F048730904BA7401A
:1005C000B04B59F410920C0410920D0410920E04CA
:1005D00010920F04E0E0F8E3099511E0A0E0B1E02B
:1005E000E6EDF3E502C005900D92A83CB107D9F7FE
:1005F00024E0A8ECB1E001C01D92AC30B207E1F7F5
:100600000E94A2130C94E9290C94000081E0089543
:1006100081E008950C94080308950C940C031F9333
:10062000CF93DF9300D000D01F92CDB7DEB74983C0
:100630005A836B833091CB0189819A81311114C027
:10064000662359F0222349F00E94D309182F682FFE
:1006500089819A810E947C0903C00E94A709182FF2
:1006600069817A81812F04C00E94D30969817A81CE
:100670000F900F900F900F900F90DF91CF911F91DF
:100680000C940D11FC01262F4081518162817381F0
:1006900084810C940F0381E00895CF93DF93EC01E4
:1006A00060E00E944203BE01DF91CF910C940D03E4
:1006B0000C9453120C944F1208950E9426080E9425
:1006C0005C032FEF84E39CE0215080409040E1F7F1
:1006D00000C000000C94E7210F931F93CF93DF938A
:1006E0008C0161E00E944203EC01B8010E940A0300
:1006F000882309F444C0B801CE010E94841F8823D6
:10070000F1F1B801CE010E94981D8823C1F1B80112
:10071000CE010E94E01E882391F1B801CE010E9413
:100720009E1C882361F1F8018281882309F1CB3571
:100730008DE5D807C1F050F4C115FCE5DF0781F065
:10074000CF3DDC45A9F40E940A0F19C0CC35EDE578
:10075000DE0761F0CD35DD4559F40E944D0E08C02D
:100760000E945D030CC00E94560E02C00E94590EEA
:10077000C801DF91CF911F910F910C94060380E087
:10078000DF91CF911F910F9108950E941B210E942C
:10079000EF030C941B1B0E94F2030E94E71B0C94B6
:1007A000212108950C94D10381E00895CF93C82F9F
:1007B0000E94D403882329F0C1FD02C0289A01C0F9
:1007C0002898CF910895209A289A0895CF93C82FFA
:1007D0000E94D2038C2F0E94D603CF91089580E00F
:1007E0000C94E6030E94E01F0C94E6030E94E01FB5
:1007F0009091CA01891721F08093CA010C94E603F5
:100800000895CF93DF93CDB7DEB72B970FB6F8944B
:10081000DEBF0FBECDBF4F83588769877A878B872E
:1008200061110E94990D9E012F5F3F4F86E0F901F3
:1008300011928A95E9F785E0FE013796D90101907A
:100840000D928A95E1F789819A814C815D81452BD2
:1008500031F09F3F31F491E08F3F19F403C091E0F4
:1008600001C090E090FF09C049815A816B817C8171
:100870008D819E810E94BA0C05C0C9010E944B0364
:100880008111F2CF2B960FB6F894DEBF0FBECDBF0D
:10089000DF91CF910895FC01808191810E94150A1A
:1008A0000895CF93882309F4A4C0C82F8238C1F4D7
:1008B0000E94E01F81FD9DC069E38091020190913B
:1008C00003010E94D6200E94BB0D2FEF81EE94E021
:1008D000215080409040E1F700C0000069E319C05A
:1008E000833801F50E94E01F80FD83C063E580919D
:1008F0000201909103010E94D6200E94BB0D2FEFB0
:1009000081EE94E0215080409040E1F700C000006B
:1009100063E580910201909103010E94E120CF9153
:100920000C94BB0D8438C1F40E94E01F82FD61C0AD
:1009300067E480910201909103010E94D6200E94F9
:10094000BB0D2FEF81EE94E0215080409040E1F705
:1009500000C0000067E4DDCF8CEF8C0F813AD0F44B
:100960006C2F80910201909103010E9456208823F0
:1009700049F06C2F80910201909103010E94E120C7
:100980000E94BB0D6C2F80910201909103010E9487
:10099000D620C5CF80E28C0F883048F4C77081E044
:1009A00001C0880FCA95EAF70E947C0DB8CFEBE52D
:1009B000EC0FE33040F4F0E0E65AFE4F808190E027
:1009C000CF910C941420E8E5EC0FE73150F4F0E0FF
:1009D000EE0FFF1FE45DFE4F80819181CF910C945B
:1009E0002A20CD3E30F08C2F0E942714CF910C94FA
:1009F000F914CF910895882309F464C0823879F4FA
:100A00000E94E01F81FF5EC069E380910201909126
:100A100003010E94D6200E94BB0D69E310C08338F9
:100A2000B1F40E94E01F80FF4DC063E58091020198
:100A3000909103010E94D6200E94BB0D63E5809136
:100A40000201909103010E94E1200C94BB0D8438B7
:100A500079F40E94E01F82FF35C067E480910201B3
:100A6000909103010E94D6200E94BB0D67E4E7CF5E
:100A70009CEF980F913A10F4682FE1CF90E2980F15
:100A8000983050F4877091E001C0990F8A95EAF789
:100A9000892F0E94820DD9CF9BE5980F933020F4C7
:100AA00080E090E00C94142098E5980F973120F4A2
:100AB00080E090E00C942A208D3E20F00E94821469
:100AC0000C94F91408951F93CF93DF93182FEB0123
:100AD0000E945104209741F08FE99FE00197F1F7C0
:100AE00000C000002197F6CF812FDF91CF911F9199
:100AF0000C94FB04893319F060E070E002C060E5FB
:100B000070E00C946305882321F00E947C0D0C9406
:100B1000BB0D0895882321F00E94820D0C94BB0D1B
:100B20000895CF92DF92EF92FF920F931F93CF938E
:100B3000DF937C01D62FC72FFC011281058102951E
:100B40000F700E94720D8823B9F01123A9F08C2F29
:100B5000807F803421F080E28D0F883068F08091B2
:100B6000E50282FD09C082E00E941B0E0E94720D08
:100B700091E0D82ED92601C0D12CCC2EC2948FE082
:100B8000C8228C2D90E08C30910508F0CFC1FC017B
:100B9000EA5AFF4F0C9444298C2F807FCF70882312
:100BA00011F0C295C07F112399F0CC2309F4AAC19A
:100BB00080E28D0F883010F0D11104C08C2F0E947C
:100BC0007C0D03C08C2F0E948C0D0E94BB0D9AC11E
:100BD0008D2F0E94FB04CC2309F4A8C180E28D0F65
:100BE000883038F1DD2329F18C2F0E94920D24C02A
:100BF0008C2F807FCF70803211F0C295C07FDD23B3
:100C000019F0D130A1F13DC08091E50282FF17C0FB
:100C1000112349F0CC2329F08C2F0E947C0D0E94D7
:100C2000BB0D80E070C180E00E94FB04CC2309F47E
:100C30007DC18C2F0E94820D0E94BB0D77C11123B4
:100C400071F0002341F0013031F40E949C0D8C2B97
:100C50000E94A40D6BC10E949C0D8C2B1DC0002313
:100C600019F0013009F462C10E94B10D25C01123B1
:100C700021F0063008F05AC10EC0053008F056C108
:100C80001BC0112361F0002331F0F701858180FF43
:100C900039C18F7085838C2F0E94830547C1002343
:100CA00059F0D93309F03FC1FFEF07EE13E0F150DF
:100CB00000401040E1F735C18C2F0E948A0536C1F3
:100CC0008C2F86958695837019F0813061F02EC146
:100CD000112321F08D2F9C2F937002C080E090E0B3
:100CE0000E9414202BC1112321F08D2F9C2F937073
:100CF00002C080E090E00E942A2020C18D2F1123A5
:100D000019F00E94271402C00E9482140E94F91454
:100D100015C18C2F837009F047C011110BC12D2F05
:100D2000229526952770220F220F6D2F6F70862F28
:100D300090E0A0E0B0E0022E04C0880F991FAA1F27
:100D4000BB1F0A94D2F7D4FF10C04FE050E060E020
:100D500070E004C0440F551F661F771F2A95D2F715
:100D6000409550956095709503C040E050E0BA0101
:100D7000C695C695C3708A019B01082B192B2A2B97
:100D80003B2BC901B801C23049F058F4C13019F009
:100D90000E949208CFC00E948008CCC00E94A40884
:100DA000C9C00E947E08C6C0112319F08C2F817023
:100DB00001C08695882309F4BDC02D2F2295269564
:100DC0002770220F220F6D2F6F70862F90E0A0E00A
:100DD000B0E0022E04C0880F991FAA1FBB1F0A94FF
:100DE000D2F7D4FF10C04FE050E060E070E004C0E4
:100DF000440F551F661F771F2A95D2F740955095CF
:100E00006095709503C040E050E0BA01C695C69564
:100E1000C3708A019B01082B192B2A2B3B2BC9017C
:100E2000B801C23049F058F4C13019F00E94570996
:100E300081C00E9445097EC00E9469097BC00E9452
:100E4000B80878C0CF70112339F08C2F0E94DE08CB
:100E50008D2F0E9483056EC08D2F0E948A058C2FD6
:100E60000E94FF0867C0D23F21F128F4D03F41F033
:100E7000D13FC1F043C0D33F19F1D43F79F03EC018
:100E8000112341F0053008F051C08C2F8F710E9462
:100E900024094CC0063008F049C0F7CF8091E50224
:100EA00082FF18C0112339F08C2F8F710E94DE0849
:100EB0003DC01123C9F38C2F8F710E94FF0836C0EB
:100EC000112329F08C2F8F710E94C9082FC00E9416
:100ED000C4082CC0112349F0CF718C2F0E94DE086A
:100EE00063E08C2F0E94000E21C081E00E941B0E47
:100EF0000230E0F082E00E941B0E18C0112331F096
:100F0000002391F28D2F0E94510410C0002399F20A
:100F1000D93349F41FEF27EE33E011502040304021
:100F2000E1F700C000008D2F0E94FB0488EF8C0DBC
:100F3000843020F40E94E01F0E94E603DD20C9F007
:100F40000E946E0D80FD15C0F70112820E94680D8F
:100F50000E94DE08C7010E94DA070E94680DDF9137
:100F6000CF911F910F91FF90EF90DF90CF900C9455
:100F7000FF08DF91CF911F910F91FF90EF90DF90CD
:100F8000CF9008950F931F93CF93DF93EC01688167
:100F900079818A810E94200A8C010E947B090E942B
:100FA0006C08B801CE010E949105DF91CF911F918D
:100FB0000F910895CF93DF93EC01988189812B8164
:100FC0003C81232B31F08F3F31F481E09F3F19F4B6
:100FD00003C081E001C080E080FD1DC0CE010E9401
:100FE0006C03811110C00E94720D8823A1F08A81C8
:100FF000882389F08091E50282FD0DC082E0DF91B7
:10100000CF910C941B0ECE010E94C207CE01DF913E
:10101000CF910C944D03DF91CF91089580E090E043
:101020000E94142080E090E00E942A200E94990DE6
:101030000E94BB0D0E942A160C94F91480910201A3
:10104000909103010E94EC200C940E080E94890DDF
:101050000C941E0892959F70963079F010F492507F
:1010600001C09A50923068F4803F69F018F4883ECD
:1010700040F409C0843F29F406C0883E20F0813F37
:1010800011F080E0089581E00895FC018081918154
:101090000E94150A0E942A080895CF93DF9300D07A
:1010A00000D01F92CDB7DEB70F900F900F900F902A
:1010B0000F90DF91CF910895CF93DF9300D000D0B0
:1010C00000D0CDB7DEB726960FB6F894DEBF0FBEC0
:1010D000CDBFDF91CF910895089508950C946D08C8
:1010E0000C946E080E9470086093020270930302D1
:1010F00080930402909305020C940E080C947208DD
:101100000F931F9300910202109103022091040299
:1011100030910502602B712B822B932B1F910F9125
:101120000C9472080F931F93009102021091030216
:1011300020910402309105026023712382239323BE
:101140001F910F910C9472080F931F93009102024C
:10115000109103022091040230910502602771274B
:10116000822793271F910F910C9472080C946D089D
:101170000E94B6086093FE017093FF018093000205
:10118000909301020C940E0860E070E0CB010C9487
:10119000B8080F931F9341E050E060E070E08A01CF
:1011A0009B0104C0000F111F221F331F8A95D2F725
:1011B000C901B8011F910F910C94B8080F931F93A8
:1011C00041E050E060E070E004C0440F551F661F2E
:1011D000771F8A95D2F78091FE019091FF01A0912F
:1011E0000002B09101028A019B01082B192B2A2BC6
:1011F0003B2BC901B8011F910F910C94B8080F93B4
:101200001F9341E050E060E070E004C0440F551FC0
:10121000661F771F8A95D2F7409550956095709517
:101220008091FE019091FF01A0910002B091010216
:101230008A019B01082319232A233B23C901B801F2
:101240001F910F910C94B8080F931F9341E050E049
:1012500060E070E004C0440F551F661F771F8A9539
:10126000D2F78091FE019091FF01A0910002B09110
:1012700001028A019B01082719272A273B27C90158
:10128000B8011F910F910C94B8080F931F93009110
:10129000FE011091FF012091000230910102602BAC
:1012A000712B822B932B1F910F910C94B8080F93E5
:1012B0001F930091FE011091FF01209100023091D7
:1012C000010260237123822393231F910F910C94B9
:1012D000B8080F931F930091FE011091FF01209118
:1012E00000023091010260277127822793271F9106
:1012F0000F910C94B80808952FE0929F800D11244F
:10130000E82FE695E695E695877051E001C0550F08
:101310008A95EAF785E0E89FF0011124E453FE4F37
:1013200020E030E070E04081CB01022E02C09695B3
:1013300087950A94E2F78170819584278523842715
:1013400081932F5F3F4F2530310569F708952FE0D6
:10135000929F800D1124682F669566956695982F4B
:10136000977085E0689FB001112440E050E080E074
:10137000FB01E40FF51FE453FE4F208130E0092EFE
:1013800002C0369527950A94E2F721703327042E80
:1013900001C0220F0A94EAF7822B4F5F5F4F45305E
:1013A000510531F70895BF92CF92DF92EF92FF92ED
:1013B0000F931F93CF93DF938C01C090FE01D090C9
:1013C000FF01E0900002F0900102809102029091F2
:1013D0000302A0910402B0910502C82AD92AEA2A80
:1013E000FB2ACFE1D0E0D701C6010C2E04C0B69590
:1013F000A795979587950A94D2F780FD04C0219709
:1014000090F7B12C07C0BC2EB8018C2F0E94201180
:101410000197A9F38B2DDF91CF911F910F91FF9031
:10142000EF90DF90CF90BF900895CF93DF93EC01C2
:101430000E94D309BE010E942011DF91CF9108952F
:101440001F93CF93DF93EB019091CB01992321F070
:10145000CB010E94150A13C0882349F0CB010E94DA
:10146000D309182F682FCE010E947C0904C0CB013C
:101470000E94A709182FBE01812F0E942011DF9121
:10148000CF911F9108951F93CF93DF93C0910602D0
:1014900016E080910702C81799F0D0E01C9FF00178
:1014A0001D9FF00D1124E85FFD4F40815181628145
:1014B0007381848195810E945C082196C770E9CF71
:1014C000DF91CF911F9108954091380250913902D8
:1014D00060913A0270913B0280913C0290913D02F2
:1014E0000C945C08EF92FF920F931F93CF93DF93BE
:1014F00080913D0282958F7009F065C080913A021B
:10150000882309F460C080910602F09007021091D0
:1015100038020091390260913B0270913C0291E0E7
:101520001F3F09F090E0C0910001D0910101292FE7
:1015300096E0E92E8F1509F446C06115710521F07A
:101540000F3F21F030E003C031E001C0322F90E0C6
:1015500030FD36C0E89EF001E99EF00D1124DF0158
:10156000A85FBD4F11963C911197301329C03C9153
:10157000311326C012963C911297311121C0139657
:101580004D915C911497461B570B4C175D07C0F4A7
:1015900080913D028F70806180933D02E35FFD4F3B
:1015A00080818F708061808388E392E00E94DA07F7
:1015B000DF91CF911F910F91FF90EF900C94430A10
:1015C00001968770B7CFDF91CF911F910F91FF9058
:1015D000EF9008959F92AF92BF92CF92DF92EF92D9
:1015E000FF920F931F93CF93DF93CDB7DEB7619731
:1015F0000FB6F894DEBF0FBECDBF8C0185E0F801B9
:10160000DE011D9601900D928A95E1F7D8011296A0
:10161000EC9090913802E091390220913B02309198
:101620003C022115310531F0EF3F31F481E09F3F5D
:1016300019F403C081E001C080E0B82FB1709B2E87
:1016400080FD47C1D8014C9111965C91119713967A
:10165000AD90BC90149788E3C82E82E0D82EF0900D
:101660003A02B501621B730B209100013091010118
:10167000FF2009F4D9C080913D026217730708F07A
:1016800095C0282F207F09F052C05E1313C0491364
:1016900011C0FE2CE1100EC08F70806180933D025E
:1016A0000E94640AC6010E94DA0780913D02F80197
:1016B00085834DC1AB2831F05F3F31F481E04F3F6E
:1016C00019F403C081E001C080E080FD03C081E027
:1016D0008E2502C080E090E0F82FF170FF2E80FF91
:1016E0001CC0809106022091070236E0821709F49F
:1016F0000BC190E0389FF001399FF00D1124E85F95
:10170000FD4F6181561306C06081461303C062819C
:10171000E61203C001968770E9CFFE2CEE2009F493
:1017200016C180913D02816080933D0254C05E13DA
:1017300006C0491304C0E11002C0F80199C0C801F5
:101740000E944508882361F1EE2051F120913D026D
:10175000822F82958F7090E0029774F0809138020A
:101760009091390298878F831986BB86AA862C8729
:10177000CE0107960E94DA0786E0F801A8E3B2E0FE
:1017800001900D928A95E1F70E94720A0E94640A04
:101790000AC05E1711F1C8010E94450881112CC0D2
:1017A000C8010E94DA07FF24F394D1C0282F207FBC
:1017B00081F77A2DB98AA88A6E2D89890E944D08F1
:1017C00088E392E00E94DA0786E0D6011D928A95AE
:1017D000E9F70E94640AF12CBAC04913DCCFE1108A
:1017E000DACFF8018583C8010E94DA0786E0D601C6
:1017F0001D928A95E9F7ABC0EE2091F220913D024F
:10180000822F82958F7090E002970CF4B5CF809173
:101810003802909139029A8389831B82BD82AC82FF
:101820002E83CE010196A6CF6217730708F044C03D
:10183000FE2CEE2009F4B4CF5E1330C049132EC045
:1018400020913D0220FD21C0822F82958F70482F6C
:1018500050E041155105C9F0F80125834F3051057D
:1018600041F08F5F982F9295907F822F8F70892BF8
:101870008583C8010E94DA0786E0F801A8E3B2E098
:1018800001900D928A95E1F73CC086E0F801A8E34B
:10189000B2E001900D928A95E1F759C0C8010E940B
:1018A0004508811169CF80913D02816080933D029E
:1018B000C8010E94DA074BC07A2DB98AA88A6E2D1A
:1018C00089890E944D0886E0D6011D928A95E9F724
:1018D00018C0EE2009F464CFC8010E944508F82E14
:1018E000882309F45DCF86E0F801A8E3B2E0019017
:1018F0000D928A95E1F788E392E00E944B040E94E2
:10190000720A0E94640A23C04D875E878D859E857A
:101910000E94150A292F22952F70223028F49F70DB
:1019200039F0811105C00BC0243028F49F7049F4B0
:10193000805E883020F0C8010E94DA079F2CF92CC5
:1019400006C0D80115969C91907F91F7F8CF8F2D06
:1019500061960FB6F894DEBF0FBECDBFDF91CF9179
:101960001F910F91FF90EF90DF90CF90BF90AF90BD
:101970009F9008951F93CF93DF93CDB7DEB72C9739
:101980000FB6F894DEBF0FBECDBF4F83588769876F
:101990007A878B879C87CE0107960E94EA0A882364
:1019A000D1F09F8188852A853B85232B31F08F3F9D
:1019B00031F481E09F3F19F403C081E001C080E071
:1019C00080FD47C04F81588569857A858B859C85C8
:1019D0000E945C083EC086E0FE013796DE0111964B
:1019E00001900D928A95E1F7FF81E8856A857B85F4
:1019F0006115710531F0EF3F31F481E0FF3F19F4DB
:101A000003C081E001C080E080FD23C02091070277
:101A100030E0C9010196877099274091060250E095
:101A200084179507F1F1F983EA837D836C8396E04F
:101A3000929FD001939FB00D1124A85FBD4FFE016E
:101A4000319601900D929A95E1F7809307020E94DA
:101A5000430A16E08091060290910702891771F1FE
:101A6000189FC0011124885F9D4F0E94EA0A8823B5
:101A700029F1E09106021E9FF0011124E85FFD4F5D
:101A80004081518162817381848195810E945C08CB
:101A90008091060290E00196877099278093060254
:101AA000D9CF0E9426081092070210920602E8E39E
:101AB000F2E086E0DF011D928A95E9F72C960FB6D9
:101AC000F894DEBF0FBECDBFDF91CF911F91089577
:101AD00080915E02859585958595089580915E0239
:101AE0008770089590915E02977081E009F480E01C
:101AF000089580918102089590918102892B8093AD
:101B000081020895809590918102892380938102BA
:101B1000089510928102089590918002892B8093FC
:101B2000800208958095909180028923809380029D
:101B3000089510928002089580915F02089508959B
:101B40000C949F0D0C94A00D9091E50292FD08C09D
:101B500090915F02981721F080935F020C94A20D80
:101B6000089580915F02882329F010925F0280E03F
:101B70000C94A20D0895CF93DF93E0910201F091B0
:101B80000301809181028083E0910201F0910301C1
:101B9000908180918002892B808380915F028823CD
:101BA00081F0E0910201F09103019081892B808303
:101BB00080910201909103010E94402081110E94B6
:101BC000B10DC0910201D091030140E250E06EE3FB
:101BD00072E0CE010E949429892B69F080E2FE0117
:101BE000AEE3B2E001900D928A95E1F7CE01DF916C
:101BF000CF910C94EC1FDF91CF9108950C949F0D21
:101C00009091E50292FD10C098E0899F9001112407
:101C1000262B20935E020E94DE0880915E0285954D
:101C2000859585950C94FE0D0C94DE0810925E024D
:101C300080E00C94FE0D20915E02809582238093BB
:101C40005E02982F977099F430E0482F082E000C10
:101C5000550B2417350759F09091E50292FD07C006
:101C60008595859585950E94FF080C94160E08951C
:101C70009091E50292FB222720F9281769F080FB5A
:101C800092F99093E5028091E4029091E5020E941E
:101C9000860E82E00C941B0E08958091E50282FB73
:101CA000882780F991E089270C94380E81E00C9404
:101CB000380E80E00C94380E6FEF7FEF80E090E0FC
:101CC0000C94D32980E090E00E94AF2921E0893E66
:101CD0009E4F09F020E0822F089582E090E00C945E
:101CE000A12983E090E00C94A129CF9384E090E0B7
:101CF0000E94A129C82F82E290E00E94A1292C2FE6
:101D000030E0A901582BCA01CF910895CF93C92F74
:101D1000682F84E090E00E94B5296C2F82E290E069
:101D2000CF910C94B529AB01BC018FE090E00C94ED
:101D3000C729AB01BC0183E190E00C94C72960E0A6
:101D400070E0CB010C94990E60E070E0CB010E9432
:101D5000930E0C949F0E69EE7EEF80E090E00E945F
:101D6000D32960E082E090E00E94B52960E083E042
:101D700090E00E94B5291092020210920302109284
:101D800004021092050260E084E090E00E94B52910
:101D900060E082E290E00E94B52960E085E090E09A
:101DA0000E94B52960E086E090E00E94B5296FEFBF
:101DB00087E090E00E94B52940E050E0BA0188E059
:101DC00090E00E94C72960E08DE090E00E94B52974
:101DD00040E050E0BA0188E190E00E94C72960E04D
:101DE00087E190E00E94B52940E050E0BA018CE123
:101DF00090E00E94C72960E070E080E290E00E94DD
:101E0000D32940E050E0BA0188E190E00E94C72960
:101E10000C94A40E0C94AB0E682F8EE090E00C9402
:101E2000B5290E94A621609390027093910280933D
:101E300092029093930260938C0270938D02809330
:101E40008E0290938F02089585B7806885BF85B70D
:101E5000806885BF089581E008950C942B0F089544
:101E60000C942F0F0C942F0F0C94320F0C942F0FF7
:101E70000C94360F0C942F0F0E94240F8CEF91E1DD
:101E80000E94D61F0E943A0F0C94380F0E94300F08
:101E90000C942F0F0E9416120C94E3030E949121C0
:101EA0000E94FB120E944A0F0E94AC1B0C94340F3C
:101EB0005F926F927F928F929F92AF92BF92CF92DA
:101EC000DF92EF92FF920F931F93CF93DF93CDB7E3
:101ED000DEB72A970FB6F894DEBF0FBECDBF0E94C3
:101EE0001013C82E81110E94110F32E8832E32E0A8
:101EF000932E00E010E0502E802F0E943A125C01D9
:101F0000F401619071904F01682679266114710483
:101F1000B1F40F5F1F4F0530110569F78FEF89830B
:101F20008A831B820E949A218160782F9D838C83F3
:101F300049815A816B818D810E9401043AC0809150
:101F4000940281FD0E944312D12CEE24E394F12CE3
:101F5000C3018E219F21892B29F10E942D0F8823F7
:101F6000A9F0DE825F82AE20BF2081E0AB2809F4B9
:101F700080E088870E949A218160782F9A878987DC
:101F80004E815F8168858A850E940104000F111FC0
:101F9000F801EE57FD4F80819181E826F926F18204
:101FA000E08207C0D394EE0CFF1CFFE0DF12D0CF1D
:101FB000B0CF81E0C11001C080E02A960FB6F8943E
:101FC000DEBF0FBECDBFDF91CF911F910F91FF906C
:101FD000EF90DF90CF90BF90AF909F908F907F90C9
:101FE0006F905F9008950E94580F0E94F01B0E940E
:101FF00017150C94F603CF93DF930E942511EC0183
:10200000811521E5920708F045C0811530E5930759
:1020100008F094C0883E910528F5803E910508F0AF
:10202000F8C0883A910570F4853A910508F07CC0B3
:102030008130910509F475C008F4E8C0049708F0F0
:10204000E8C0E4C08F3B910508F0E0C0C85AD0E07A
:10205000CC0FDD1FC35ADE4F0990D881C02DCE01B1
:102060009464D8C0811540E2940758F4811551E07A
:10207000950708F0CEC08D3E910508F4C7C0906565
:10208000C9C0C11580E4D80708F4C0C0DF70CE0114
:10209000906AC0C0811525E59207A8F4811534E542
:1020A000930708F095C0811543E5940708F07BC0BD
:1020B000811552E5950708F061C0D82FCC27CE01D5
:1020C000816F906AA7C0C11589E5D807A0F4C11532
:1020D00028E5D20708F082C0C11536E5D30708F01D
:1020E00095C08C2F0E94B9118F7190E0D82FCC270A
:1020F000CE0190628FC0C1154AE5D40708F474C0C0
:10210000CE0190568115904208F080C08D2F8F71BE
:102110000E94B911DD27D0628F71AE01582BCA0120
:1021200079C081E090E076C0C55AD0E0C557DE4F57
:102130008881C82FD0E0CE0190646CC074E0969581
:1021400087957A95E1F7282F23703C2F337081E033
:1021500090E002C0880F991F3A95E2F79C68AC01A5
:10216000522B9A019C2F9F709695969550E2959FC1
:10217000E0011124C9018C2B9D2B4CC08370992741
:1021800021E030E002C0220F331F8A95E2F79C2F36
:102190009695969580E2989FE0011124C22BD32B4F
:1021A000CE019C6837C08370992721E030E002C0DF
:1021B000220F331F8A95E2F79C2F9695969540E261
:1021C000949FE0011124C22BD32BCE019A6822C028
:1021D000D82FCC27CE01846F906A1CC0DC2FCC276F
:1021E000CE01806F906A16C08C2F8F700E94B9113B
:1021F00094E0D695C7959A95E1F7CF70D0E0DC2FA3
:10220000CC27D0699E01282BC90104C080E090E052
:1022100001C0CE01DF91CF9108952BE4829FC001D0
:102220001124FC012FE0729FE00DF11D1124E60F37
:10223000F11DEE0FFF1FE852FF4F85919491089515
:102240000E940D110E94FB0F08958238910569F1DB
:10225000B0F48133910509F46DC048F489329105D9
:1022600009F463C08A32910509F469C00895853381
:10227000910509F455C089339105B9F00895833E5D
:10228000910569F138F4803E9105B1F0823E9105E7
:1022900009F10895863E9105A9F1873E9105B9F1AE
:1022A000843E910509F064C023C02091E40220FD22
:1022B0004FC021FD4DC008958091E40280FD44C0CF
:1022C0008091E50280FF44C08091E40284FD42C019
:1022D00083EE4DC08091E40282FF38C0F5CF80913B
:1022E000E40282FD33C08091E50280FD31C0ECCF75
:1022F0008091E50281FF32C08091E40284FD2AC012
:1023000087EE35C08091E40283FF26C0F5CF80912F
:10231000E40283FD21C08091E50281FD1FC0ECCF66
:102320008091E40285FD1CC01DC08091E40285FD02
:1023300019C016C08091E40286FD16C017C08091B6
:10234000E40286FD13C010C089E311C082EE0FC005
:1023500080EE0DC080E00BC086EE09C084EE07C0A1
:1023600089E205C085E303C08AE201C081E390E011
:1023700008959091E40292FF0DC0282F2871283013
:1023800019F4877F846006C0282F2471243011F44B
:102390008B7F886093FF0DC0282F2871283119F496
:1023A000877E846106C0282F2471243111F48B7E2E
:1023B00088612091E50220FF0DC0382F3871383038
:1023C00019F4877F816006C0382F3171313011F4E4
:1023D0008E7F886021FF0DC0282F2871283119F4C5
:1023E000877E816106C0282F2171213111F48E7EF4
:1023F000886194FD877E089580E008950C945C0EBA
:102400000E9410138FE39CE90197F1F700C00000D0
:102410000E94101380E00E943A1280FF04C00E94C4
:10242000FE110C94E72108950C9400120E94620E94
:10243000811102C00E940A0F0E946D0E80939402C7
:102440000E94750E9093E5028093E4020E9414129C
:102450000E94710E682F70E080E090E00E947E087C
:102460006091FE017091FF01809100029091010244
:102470000C94B608E82FF0E0EE0FFF1FE051FD4F7F
:10248000808191810895089580EA8A95F1F70895F1
:1024900000C008950C94441208950C944C120C94AE
:1024A0004D120C944C120C945112F894E82FE295B2
:1024B000EF70F0E031A1282F2F7081E090E001C093
:1024C000880F2A95EAF7982F9095932391A392A1CC
:1024D000892B82A3789408950F931F93CF93DF9352
:1024E000CDE9D1E089918F3F11F00E94551281E032
:1024F000C23AD807B9F7CEE8D1E00DE911E08991E9
:102500008F3F11F00E9455120C171D07C1F7DF9184
:10251000CF911F910F910895BF92CF92DF92EF92CA
:10252000FF920F931F93CF93DF938C01C62FD0E0C0
:10253000CE0183569E4F6C01FC0190819F3F09F4B0
:1025400050C0B62EF894E92FE295EF70F0E081A12B
:102550009F7021E030E001C0220F9A95EAF7822BAC
:1025600081A382A12095282322A378940E94481257
:10257000EEE8F1E04DE951E021E030E0E12CF12C12
:1025800061916F3F89F0A62FA295AF70B0E0909651
:102590008C9190E06F7002C0959587956A95E2F7EF
:1025A00080FD02C0C90102C080E090E0E82AF92A5B
:1025B000220F331F4E175F0719F7F60180818F3FF7
:1025C00011F00E94551261E0E114F10409F460E099
:1025D0008B2D0E944A12CC0FDD1FC00FD11FF98234
:1025E000E882DF91CF911F910F91FF90EF90DF90E4
:1025F000CF90BF9008950E946C128AE0E0EFF2E065
:10260000DF01982F1D929A95E9F7E6EEF2E0DF01DF
:102610001D928A95E9F785E00E945B130C9458039C
:10262000FF920F931F93CF93DF93CDB7DEB72A9717
:102630000FB6F894DEBF0FBECDBF8E010F5F1F4FE8
:102640008AE0F80111928A95E9F7F12C6F2DC80103
:102650000E948C12F394F5E0FF12F8CF4AE050E0AC
:10266000B80186EE92E00E949429FF24F39400972B
:1026700009F4F12C892B41F08AE0F801A6EEB2E0D2
:1026800001900D928A95E1F72F2D45E060EF72E001
:1026900086EE92E00E945C130E945A038F2D2A96C8
:1026A0000FB6F894DEBF0FBECDBFDF91CF911F9163
:1026B0000F91FF9008950895FF920F931F93CF936A
:1026C000DF93F82E092F162FD72FC42F222349F07E
:1026D00081E0809397020E949A21909396028093C2
:1026E0009502809197028823D9F08091950290916C
:1026F00096020E94B221059798F0EF2DF02FA12F9E
:10270000BD2F80E090E04C2F50E08417950734F403
:10271000219131912D933D930196F7CF109297021D
:10272000DF91CF911F910F91FF9008950E94B223E6
:102730000E944E0F0C94BE230E94C2230E94F30FEE
:102740000C94DC230E9438210E9499230E943C0FA4
:102750000E9496130E949C130E94460FFBCF80910B
:102760009E0280FF06C06091090170E0660F771F2E
:1027700026C081FF04C06091090184E005C082FF8A
:1027800007C06091090188E0689FB001112417C05B
:1027900090919D029923D1F060910801961788F7D6
:1027A0002091090188E0289F90011124929FA001A7
:1027B000939F500D112470E0CA010E940E296038C9
:1027C000710540F46115710519F406C068E070E008
:1027D000862F08958FE7089581E0089580919E02E5
:1027E00080FF08C06091050170E07595679575954B
:1027F000679521C081FF06C06091050170E0759565
:10280000679519C082FF04C06091050170E010C097
:1028100090919C02992399F0609104019617A0F77A
:1028200080910501899FC001112470E00E940E294A
:102830006038710540F46115710519F406C061E056
:1028400070E0862F08958FE7089581E008958D3E0A
:1028500021F40E94AF13819504C08E3E29F40E949A
:10286000AF138093A20208958F3E21F40E94AF130C
:10287000819504C0803F29F40E94AF138093A10288
:102880000895893F19F40E94EE1305C08A3F31F480
:102890000E94EE1381958093A30208958B3F21F44B
:1028A0000E94EE13819504C08C3F29F40E94EE1320
:1028B0008093A40208959FE0980F983078F421E067
:1028C00030E0A90102C0440F551F9A95E2F7CA01F2
:1028D0009091A002892B8093A00208958D3F21F44E
:1028E00080919E0281600BC08E3F21F480919E02F8
:1028F000826005C08F3F29F480919E02846080939E
:102900009E0208958D3E39F49091A20297FF35C042
:102910001092A20259C08E3E29F49091A20219167B
:10292000BCF32BC09091A1028F3E29F497FF25C0E4
:102930001092A10249C0803F19F41916CCF31DC0B2
:102940009091A302893F29F41916BCF41092A302B6
:102950003BC08A3F19F497FF10C0F8CF8B3F39F482
:102960009091A40297FF09C01092A4022DC08C3F41
:1029700021F49091A4021916BCF39FE0980F9830AF
:1029800080F421E030E0A90102C0440F551F9A9560
:10299000E2F7CA0180959091A00289238093A0025A
:1029A00013C08D3F21F480919E028E7F0BC08E3F1D
:1029B00021F480919E028D7F05C08F3F29F4809184
:1029C0009E028B7F80939E028091A102811106C09E
:1029D0008091A202811102C010929D028091A302F7
:1029E000811106C08091A402811102C010929C0244
:1029F00008950E949A212091A102211104C02091E2
:102A0000A202222321F090939B0280939A022091AC
:102A1000A302211104C02091A402222321F090934B
:102A20009902809398028FE992E00C940620EF922D
:102A3000FF920F931F93CF93DF9300D000D000D06D
:102A4000CDB7DEB786E0EFE9F2E0DE011196019046
:102A50000D928A95E1F7E090A102F090A202009118
:102A6000A3021091A4021092A1021092A20210924D
:102A7000A3021092A402E11003C0FF2009F45DC07C
:102A800080919A0290919B020E94B221AC01909198
:102A90009D02992339F020910A0130E0241735076F
:102AA00058F04BC020910B018AE0289F900111241F
:102AB0002417350718F041C09F3F19F09F5F90938E
:102AC0009D02EE2061F00E94AF131E1414F09FEFE0
:102AD00001C091E0989F902D11249093A102FF20B6
:102AE00061F00E94AF131F1414F09FEF01C091E03A
:102AF000989F902D11249093A2023091A10233232C
:102B0000E1F02091A2022223C1F045EB3403C00181
:102B10001124992319F09093A10203C081E08093BE
:102B2000A10235EB2303C0011124992319F09093DE
:102B3000A20203C081E08093A202011103C011230D
:102B400009F45DC080919802909199020E94B2218F
:102B5000AC0190919C02992339F02091060130E05C
:102B60002417350758F04BC0209107018AE0289FB1
:102B7000900111242417350718F041C09F3F19F028
:102B80009F5F90939C02002361F00E94EE13101649
:102B900014F09FEF01C091E0989F902D1124909325
:102BA000A302112361F00E94EE13111614F09FEF9F
:102BB00001C091E0989F902D11249093A402309130
:102BC000A3023323E1F02091A4022223C1F045EBBC
:102BD0003403C0011124992319F09093A30203C078
:102BE00081E08093A30235EB2303C00111249923D4
:102BF00019F09093A40203C081E08093A402809115
:102C0000A10281110BC08091A202811107C08091A5
:102C1000A302811103C08091A40281110E94F914C2
:102C2000EB82FC820D831E8386E0FE013196AFE9C4
:102C3000B2E001900D928A95E1F726960FB6F894CE
:102C4000DEBF0FBECDBFDF91CF911F910F91FF90DF
:102C5000EF900895EFE9F2E086E0DF011D928A959A
:102C6000E9F710929D0210929C0210929E02089524
:102C7000EF92FF920F931F93CF93DF938B01682FF7
:102C800011110AC0442329F0E82FF0E0E55EFC4F63
:102C90006491762F862F75C0212F30E0E82FF0E069
:102CA000442321F0E55EFC4FE491F0E046E0049F10
:102CB000C0011124CFEFD0E0BE010E94FA284BEAF8
:102CC0004603C001479F900D1124800F911D800F76
:102CD000911D982F990F890FAE01421B530B4E9FE8
:102CE000D0014F9FB00D5E9FB00D11249B2F189FF8
:102CF000A0011124452F55278E01041B150B0E9F93
:102D0000A0010F9F500D1E9F500D11247E01E81A47
:102D1000F108E29E8001E39E100DF29E100D112439
:102D2000212F3327C21BD30BCE9F9001CF9F300D95
:102D3000DE9F300D112462307105A9F048F4611551
:102D4000710569F061307105C9F48B2F752F0DC0C5
:102D50006430710581F058F06630710579F47E2F8A
:102D60008B2F932F0DC0832F7B2F9E2F09C08E2F6B
:102D70007B2F952F05C08E2F732F02C07E2F852F9E
:102D8000692FDF91CF911F910F91FF90EF900895E0
:102D900041E00E943816089508950E94C8160895CB
:102DA000CF93DF93762FE901682F842F0E94CD16F1
:102DB000798368838A83DF91CF9108958091FA02A5
:102DC000282F269530E02115310519F48170826095
:102DD00005C02532310524F0817088648093FA02A1
:102DE000089588E090E00C94A929CF92DF92EF92A9
:102DF000FF926B017C010E94DE16B701A60188E0FC
:102E000090E0FF90EF90DF90CF900C94C729EAEF0D
:102E1000F2E083E0808311828FEF828383831482C8
:102E200060817181828193810C94F5168091FA0200
:102E300080FF02C08695089580E008959091FE027B
:102E4000933018F49F5F9093FE02882351F06091B5
:102E5000FA027091FB028091FC029091FD020C94A9
:102E6000F516089581E00C941E179091FE029923A7
:102E700019F091509093FE02882351F06091FA026C
:102E80007091FB028091FC029091FD020C94F5166A
:102E9000089581E00C94351770E00C946D1D6091DD
:102EA00010018091FA0280FF0AC080910F0123E097
:102EB000829FC001112481509D4F0C944C1780912A
:102EC000110190911201891780F7E82FF0E09F011E
:102ED000220F331FE20FF31FE150FD4F11821082CA
:102EE00012828F5FF0CF9091FA0290FF16C09091FE
:102EF000110120911201921770F4E92FF0E0DF0127
:102F0000AA0FBB1FEA0FFB1FE150FD4F81836083B7
:102F100042839F5FF0CF0C944F170895CF93DF93B8
:102F200000D01F92CDB7DEB79091FA0290FF0AC091
:102F30009E012F5F3F4F0E94D0164B8169818A818D
:102F40000E9473170F900F900F90DF91CF9108950B
:102F5000CF93DF93EC01EC81F0E0EA5EFD4F44910A
:102F6000EAEFF2E0628181810E948E178C818F5F8F
:102F70008C83DF91CF910895CF93DF93EC01EAEF3B
:102F8000F2E0438162818C810E948E178C818F5F79
:102F90008C83DF91CF9108950F931F93CF93DF938D
:102FA00000D01F92CDB7DEB78C018091A5028111B0
:102FB0000AC09E012F5F3F4F4FEF6FEF0E94D01668
:102FC0008A818093A502F8018481813051F028F034
:102FD000823061F44091A5020AC08091A50240E0D0
:102FE00007C06091A50240E080E003C040E080E0BF
:102FF00060E00E947317F801848190E0019663E01D
:1030000070E00E940E2984830F900F900F90DF9143
:10301000CF911F910F910895AF92BF92CF92DF92FF
:10302000EF92FF920F931F93CF93DF9300D01F92E5
:10303000CDB7DEB7182FF62E042FE22E9091FA02AC
:1030400090FF6DC0E92FE695AE2FB0E0AE55BE4FB4
:103050008C918093B1029E7F923061F49E012F5F2C
:103060003F4F812F0E94D0164B8169818A810E9437
:10307000731743C0823019F40091FD023EC08630C0
:1030800019F41091FB0239C08930D9F38931A9F5BF
:10309000E9518E2F8170D82EE695F0E0EA5EFC4F64
:1030A000A590B490C12CBB2460911301C61618F5ED
:1030B0002C2D30E0A29EC001A39E900DB29E900DDB
:1030C000112470E00E94FA28812FD11002C0860FCF
:1030D00001C0861B90911101290F311DA901440FD8
:1030E000551F240F351F21503D4F402F6F2D0E943B
:1030F000D016C394D9CF0E944F171093FB02F092C1
:10310000FC020093FD02EE2051F06091FA027091F2
:10311000FB028091FC029091FD020E94F5160F9037
:103120000F900F90DF91CF911F910F91FF90EF9033
:10313000DF90CF90BF90AF900895EAEFF2E09181D9
:10314000282F4381628188E0890F0C940C1881E05C
:103150000C949D18EAEFF2E09181282F438162815F
:1031600088EF890F0C940C1881E00C94AA18EAEFF0
:10317000F2E0628128E0620F08F46FEF282F4381AC
:1031800081810C940C1881E00C94B718EAEFF2E0FE
:10319000628128E0621B08F460E0282F438181816E
:1031A0000C940C1881E00C94C618EAEFF2E043810D
:1031B00028E0420F08F44FEF282F628181810C94A0
:1031C0000C1881E00C94D518EAEFF2E0438128E076
:1031D000421B08F440E0282F628181810C940C1876
:1031E00081E00C94E41820E00C940C18FF920F93EB
:1031F0001F93CF93DF93EC01F12C0FEF10E0609160
:103200001301F616F0F4809111012F2D30E0280FF4
:10321000311DC901880F991F280F391F21503D4FBB
:1032200070E0C8010E940E29962F8C814091FD020A
:103230006091FC02F99E800D11240E94D016F39437
:10324000DECF0E944F179A818C8190FF02C08F5F62
:1032500001C081508C83DF91CF911F910F91FF901E
:103260000895AF92BF92CF92DF92EF92FF920F93A9
:103270001F93CF93DF93FC01828180FF02C00FEF89
:1032800001C001E010E044E5A42E8091130118175D
:1032900008F043C080911101C12ED12CE601C80F66
:1032A000D11DCE01880F991FC80FD91FC150DD4F06
:1032B000198218821A8234E0E32EF12CB12C80910D
:1032C000A7028B0D85352CF06A2D0E94EC28892FE2
:1032D00005C087FF03C090911301890F082E000CD1
:1032E000990BC816D90691F48091FD028E9DA0011C
:1032F0008F9D500D112455954795559547959E01E5
:103300006091FC028091FB020E94D016B00EF1E0A9
:10331000EF1AF108A1F61F5FB8CF0E944F178091F6
:10332000A702013031F4811102C080911301815054
:1033300007C090E001966091130170E00E940E2991
:103340008093A702DF91CF911F910F91FF90EF9093
:10335000DF90CF90BF90AF900895CF9380911101EF
:1033600090911201891770F4E82FF0E09F01220F6D
:10337000331FE20FF31FE150FD4F118210821282C2
:103380008F5FF0CFC0E060911301C617C0F5EC2F3E
:10339000F0E070E0CF010E940E2920911101820F10
:1033A0002091A602022E000C330B90E0E217F307E7
:1033B000CCF020910E01022E000C330B2E173F078C
:1033C0008CF09C01220F331F820F931F9C01215010
:1033D0003D4F4091FD026091FC028091FB020E94F2
:1033E000D0160BC0FC01EE0FFF1F8E0F9F1FFC01BC
:1033F000E150FD4F118210821282CF5FC4CF0E9434
:103400004F1720910D018091A602820F8093A60292
:1034100090910E01920F90930E0119165CF4082EF4
:10342000000C990B4091130150E041505109841751
:1034300095071CF0219520930D01CF9108958F924F
:103440009F92AF92BF92CF92DF92EF92FF920F9333
:103450001F93CF93DF938C01FC014481C42FD0E0F4
:103460009E01DE010E9452299B01AC010E94682945
:103470006B017C01E0E2F0E0EC1BFD0BA5E5B0E0A8
:103480009B01AC010E9468294B015C019F01DF0197
:103490000E944A299B01AC010E9473299B01AC0147
:1034A0002C0D3D1D4E1D5F1DC501B4010E9422293A
:1034B000C22FD22F2A3228F4F3E02F9F900111243B
:1034C0000DC025E530E02C1B3109C901880F991F7B
:1034D000280F391F37FF02C02F5F3F4F35952795C3
:1034E000C22FC095F12C85E5E82EED1A80911301CD
:1034F000F816C8F4F1FC02C08E2D01C08D2F9091FA
:1035000011012F2D30E0290F311DA901440F551F46
:10351000240F351F21503D4F4C2F6091FC020E941B
:10352000D016F394E3CF0E944F17F80184818111E4
:1035300002C091E003C0803219F49FEF90930C0118
:1035400090910C01890FF8018483DF91CF911F9135
:103550000F91FF90EF90DF90CF90BF90AF909F9032
:103560008F9008950F931F93CF93DF93EC0100E0AA
:1035700010E080911301282F30E00217130724F583
:10358000909111019801290F311DA901440F551F78
:10359000240F351F21503D4F869590E04C81081730
:1035A00019071CF4442331F002C0411103C04091BB
:1035B000FD0201C040E06091FC028091FB020E948C
:1035C000D0160F5F1F4FD5CF0E944F178C8190E010
:1035D0000196817099278C83DF91CF911F910F9174
:1035E0000895EAEFF2E080818E7F808360817181AF
:1035F000828193810E94F5161092B2022FEF80E72C
:1036000092E0215080409040E1F700C000000C940F
:103610004F17EAEFF2E080818E7F80831092B20232
:103620002FEF80E792E0215080409040E1F700C00A
:1036300000000C944F171092B2028091AF028111DA
:103640000AC081E08093AF028091FA02817080937A
:10365000AE020C94091B08956091FA02669570E021
:103660004BE050E084E191E00E948729892B19F416
:1036700081E08093B2020E949A219093A9028093E4
:10368000A80208959091FA0290FF35C091708111BF
:1036900002C0926006C0853210F0986402C0880FA4
:1036A000982B9093FA02662351F06091FA02709180
:1036B000FB028091FC029091FD020E94F516609140
:1036C000FA02669570E04BE050E084E191E00E94E0
:1036D0008729892B19F01092B20202C00E942C1B7C
:1036E00081E08093AB024091FD026091FC028091E9
:1036F000FB020C94F3180895682F9091FA029695A6
:1037000081E0890F853208F081E00C94421B81E052
:103710000C947C1B682F9091FA0296958FEF890F7D
:1037200009F484E20C94421B81E00C948A1B61E052
:103730000C94421BEAEFF2E08081816080838695E1
:103740000C94971B8091FA0280FD0C94F11A0C9452
:103750009A1B60E00C94421B8091B00281112EC034
:103760000E94620E811104C00E940A0F0E94071776
:103770000E94F1166093FA027093FB028093FC02A0
:103780009093FD026E7F61F40E9407170E94F1166C
:103790006093FA027093FB028093FC029093FD0207
:1037A0000E94DE161092B2028091FA0280FF03C0DE
:1037B00086950E94A91B81E08093B0020895EAEFEC
:1037C000F2E080818160808386950C94A91B109221
:1037D000AF028091AE0281110E94DF1B0C942C1B62
:1037E0000F931F93CF93DF938091B202882309F444
:1037F00085C08091B102E091FA02E695E81BE09362
:10380000AA02823049F4F0E0EE5EFD4FE491CE2F43
:10381000D0E008EA17E149C0863049F4F0E0E15F02
:10382000FD4FE491CE2FD0E00CEB17E13EC0893084
:1038300051F4E695F0E0E45FFD4FE491CE2FD0E047
:1038400006EF18E132C08F3051F4E695F0E0E75F03
:10385000FD4FE491CE2FD0E001E319E126C0853180
:1038600049F4F0E0EA5FFD4FE491CE2FD0E00DEA9D
:1038700019E11BC0883181F0833239F4E4E0F2E0D1
:10388000C591D4910CEC17E110C0843251F4C4EF0F
:10389000D1E002EB1AE109C0C8E2D0E00FE11AE181
:1038A00004C0C0EDD7E00CEC16E18091AB02882398
:1038B00061F01092AB020E949A219093A90280932A
:1038C000A8021092AD021092AC020E949A21E091DF
:1038D000A802F091A9028E1B9F0B8F3F9F4770F4A7
:1038E000EC0FFD1FF093A902E093A80288EA92E092
:1038F000F801DF91CF911F910F910994DF91CF9142
:103900001F910F910895882311F0FA0101C0FB0166
:103910000994CF93DF93C82FD62F0E9416178C17C8
:1039200040F00E9416178D1720F4DF91CF910C9470
:10393000871B8C2FDF91CF910C94971B1F93CF93F4
:10394000DF93FB0112811111C3C0EC010E94790DBC
:103950008272CD3CFCE5DF0709F49AC0A8F5C73CAC
:10396000ECE5DE0709F476C0A8F4C43C9CE5D90771
:1039700009F45FC028F4C33CDC4509F457C054C0C7
:10398000C53C9CE5D90709F459C0C63CDC4509F49F
:103990005CC04AC0CA3CFCE5DF0709F46AC050F4C9
:1039A000C83CECE5DE0709F45AC0C93CDC4509F423
:1039B0005BC03AC0CB3C9CE5D90709F45FC0CC3C66
:1039C000DC4509F460C030C0C23DFCE5DF0709F406
:1039D0006FC088F4CF3C9CE5D90709F460C008F4B7
:1039E0005CC0C03DFCE5DF0709F45CC0C13DDC45BF
:1039F00009F45BC019C0C53D9CE5D90709F460C056
:103A000050F4C33DFCE5DF0709F455C0C43DDC4577
:103A100009F454C009C0C63D9CE5D90709F455C056
:103A2000CE35DD4509F454C011E052C00E94A21BFE
:103A30004FC044E95BE167E87BE104C047E85BE134
:103A400064E97BE10E94831C43C044EB58E167EAD0
:103A500078E1F8CF47EA58E164EB78E1F3CF42ED43
:103A600058E163EC78E1EECF43EC58E162ED78E1A8
:103A7000E9CF40EF58E161EE78E1E4CF41EE58E163
:103A800060EF78E1DFCF49E457E162E377E1DACF35
:103A900042E357E169E477E1D5CF81E017C065E003
:103AA00082E010C068E086E00DC06EE089E00AC0E8
:103AB00064E18FE007C067E185E104C088E106C0EA
:103AC00062E289E10E94891C03C083E20E94971B85
:103AD000812FDF91CF911F910895869A21B32F7B7B
:103AE00031B330644FB7F894FC01CB01880F991FB4
:103AF000680F791F6E0F7F1FE617F70789F0819116
:103B000098E031BB000000C087FF21BB880F000098
:103B100000C000C000C021BB00C09A9591F7ECCF57
:103B20004FBF8FE594E00197F1F700C000000895C2
:103B3000CF93DF93EC01FB018281882309F43CC120
:103B4000C430FDE5DF0760F4CB3F9CE5D90788F47E
:103B50009E0122503C452431310508F02EC109C098
:103B6000C236EDE5DE0729F0C63AFDE5DF0709F0CC
:103B700024C10E94750E9093E5028093E402C13146
:103B80008CE5D80709F4C6C008F042C0C930ECE59E
:103B9000DE0709F49BC000F5C5308CE5D80709F4B1
:103BA00085C078F4C330ECE5DE0709F478C008F08E
:103BB0007AC0C230DC4509F0F5C08091E402816032
:103BC000EFC0C7309CE5D90709F478C008F07AC087
:103BD0008091E4028061E4C0CD30FCE5DF0709F4A8
:103BE00087C058F4CB309CE5D90709F479C008F0B8
:103BF0007BC08091E40288606FC0CF30FCE5DF07B6
:103C000009F480C008F082C08091E402877FC8C0B8
:103C1000CE3F9CE5D90709F471C000F5C531FCE53C
:103C2000DF0709F485C068F4C3319CE5D90709F4BE
:103C300075C008F095C00E9426088091E4028F7735
:103C4000AFC0CC3FFCE5DF07A9F108F054C0CB3F83
:103C5000DC4509F0A7C08091E50240C0C230EDE527
:103C6000DE0709F489C058F4C1158DE5D80709F4B9
:103C70005AC008F069C08091E50282602FC0C23648
:103C8000EDE5DE0709F47CC0C63AFDE5DF0709F47F
:103C900081C0C330DD4509F085C080E06EC08091F1
:103CA000E40282607DC08091E40216C08091E4024B
:103CB000886076C08091E50282604FC08091E40206
:103CC00080626EC08091E40280646AC00E9426080F
:103CD0008091E402806864C0846062C081603DC0FD
:103CE0008091E4028E7F5CC08091E4028D7F58C099
:103CF0008091E40216C08091E50218C08091E5022F
:103D00008D7F2BC08091E4028F7E4AC08091E402B7
:103D10008F7D46C08091E4028F7B42C08091E40297
:103D2000877F8B7F3DC08091E5028D7F8E7F15C0A0
:103D30008091E40282FB222720F991E0922790FBF8
:103D400082F990FB83F92CC08091E502982F909521
:103D500091708E7F892B90FB81F98093E50222C0C0
:103D60000E9426088091E40287FB222720F991E037
:103D7000922790FB87F914C081E00E940C0F12C0BB
:103D80008091E40284FB222720F991E0922790FBA6
:103D900084F906C08091E402982F909590FB80F9F9
:103DA0008093E4028091E4029091E5020E94860EE5
:103DB0000E94260880E001C081E0DF91CF91089544
:103DC000CF93DF9386319C4541F5EB010E94790D3D
:103DD000982F8A812091020130910301882379F084
:103DE0009A7A81E009F480E08093B302911102C0D5
:103DF00069E201C065E3C9010E94D6200AC0809132
:103E0000B302811102C069E201C065E3C9010E94E9
:103E1000E1200E94BB0D80E001C081E0DF91CF91E5
:103E200008950F931F93CF93DF93C42FD22FFC01DC
:103E300082818823C9F04093B6020E949A21909310
:103E4000B5028093B40280E28C0F883008F057C02E
:103E5000C77081E001C0880FCA95EAF7DF91CF9162
:103E60001F910F910C9483058091B602481330C0C6
:103E70008091B4029091B5020E94B221883C9105D4
:103E800038F510E21D0FCD17B9F080E28C0F8830A5
:103E900040F4C77081E001C0880FCA95EAF70E941C
:103EA0008A05183028F581E09D2F977001C0880F92
:103EB0009A95EAF70E948305802F0E947A051830B0
:103EC000F0F4D77081E001C0880FDA95EAF70AC0F4
:103ED00080E28C0F883098F4C77081E001C0880FB1
:103EE000CA95EAF7DF91CF911F910F910C948A0543
:103EF000802FDF91CF911F910F910C947A05DF9164
:103F0000CF911F910F9108950F939C01CB01243FF6
:103F10004CE5340731F188F4293DFCE53F07D9F041
:103F20002A3D4CE5340779F1283D3C45A9F506E2E8
:103F300021EE41EE68ED7CE52BC0263FFCE53F0716
:103F4000E1F0A8F0273F3C4539F507E225EE46EEC3
:103F500067EF7CE51DC007E225EE45EE69ED7CE5E7
:103F600017C006E221EE40EE64EF7CE511C007E2E7
:103F700025EE44EE65EF7CE50BC006E221EE42EE55
:103F800066EF7CE505C008E221E045EE6AED7CE5E0
:103F90000E94111F80E008C0FC018281882319F073
:103FA0001092B60201C081E00F9108959093C9016B
:103FB0008093C80108959093BC028093BB0208953A
:103FC000E091BB02F091BC02309721F00190F081AA
:103FD000E02D099480E00895E091BB02F091BC02CD
:103FE000309799F020912B01222359F02091E4027F
:103FF00027FF07C0DC012C9111962C93119726E026
:104000002C930280F381E02D09940895E091BB0286
:10401000F091BC02309739F022E0DC012C9304804F
:10402000F581E02D099408952091B9023091BA02EA
:104030002817390771F09093BA028093B902E09182
:10404000BB02F091BC02309721F00680F781E02D91
:10405000099408952091B7023091B80228173907C2
:1040600071F09093B8028093B702E091BB02F09197
:10407000BC02309721F00084F185E02D0994089569
:10408000FC01329680912B01882331F08091E4026B
:1040900087FF02C09EE101C096E080E0915028F0C9
:1040A00021912223D9F38F5FF9CF0895662351F12F
:1040B00020912B012223E9F02091E40227FF19C06F
:1040C000462F4695469546954E31E0F4677021E0BF
:1040D00030E002C0220F331F6A95E2F7FC01E40FC3
:1040E000F11D828190E02823392381E0232B69F49C
:1040F00009C0FC01329608962191621729F0E81751
:10410000F907D1F780E0089581E008959C01FC0152
:1041100032969FEF80E04191461789F09F3F19F456
:10412000411101C0982F8F5F8630A9F79F3F39F06A
:10413000F901E90FF11D97FDFA956283089508953D
:104140009C012A5F3F4FFC014281461301C012824D
:10415000019682179307B9F70895262F269526957D
:1041600026952E3168F4FC01E20FF11D677021E005
:1041700030E001C0220F6A95EAF78281282B228362
:104180000895262F2695269526952E3170F4FC014C
:10419000E20FF11D677021E030E001C0220F6A9547
:1041A000EAF72095828128232283089520912B010C
:1041B000222329F02091E40227FD0C94AD200C94D9
:1041C000862020912B01222329F02091E40227FD53
:1041D0000C94C1200C94A02020912B01FC0132965C
:1041E000222331F08091E40287FF02C08EE101C0FA
:1041F00086E0DF011D928A95E9F7089508950C94F1
:10420000FE2083E08093BD020C94FF20811102C048
:1042100081E001C082E08093BD020C94FF200C94E9
:10422000062181E08093BD020C94FF200C941121A3
:1042300008950C9418210C9419210C9418210C94B5
:1042400018210C941821CF930E941F210E94101353
:104250000E941D21C0E08C2F0E943A12892B29F464
:10426000CF5FC530C1F780E001C081E0CF910895F4
:1042700008951F920F920FB60F9211248F939F9360
:10428000AF93BF938091BE02811113C08091FB0355
:104290009091FC03A091FD03B091FE034196A11DF6
:1042A000B11D8093FB039093FC03A093FD03B09397
:1042B000FE03BF91AF919F918F910F900FBE0F9012
:1042C0001F90189580910304843031F10E94C5033A
:1042D0001092BE0220E488E190E00FB6F894A89511
:1042E000809360000FBE2093600083B7817F84605D
:1042F00083BF83B7816083BF7894889583B78E7FAF
:1043000083BF0FB6F894A895809160008861809370
:104310006000109260000FBE08950E9426080C9461
:10432000CB0382E084BD93E095BD9AEF97BD809367
:104330006E0008952FB7F8948091FB039091FC03D1
:10434000A091FD03B091FE032FBF08952FB7F894FD
:104350006091FB037091FC038091FD039091FE033B
:104360002FBF08959C014FB7F8948091FB03909163
:10437000FC03A091FD03B091FE034FBF821B930B82
:10438000089578941F920F920FB60F9211248F9375
:104390009F93AF93BF938091FB039091FC03A091F7
:1043A000FD03B091FE030196A11DB11D8093FB0397
:1043B0009093FC03A093FD03B093FE03BF91AF91D4
:1043C0009F918F910F900FBE0F901F90189581E0D5
:1043D0008093E00080E28093D8001092C9008FE1C2
:1043E0009EE40197F1F700C0000087E090EBDC014C
:1043F00080930C0490930D04A0930E04B0930F04CB
:104400009CE088E10FB6F894A895809360000FBEF9
:1044100090936000FFCF8091E2020895089522E01A
:104420002093E9002FEF3091E800215035FD06C0C0
:1044300035ED3A95F1F700002111F5CF2091E80014
:1044400025FF0BC040E050E066E070E00E944E2483
:104450008091E8008E778093E8000895CF93DF93F2
:1044600020912B01222339F02091E40227FF03C081
:1044700060E222E002C068E021E02093E9002FEF33
:104480003091E800215035FD06C035ED3A95F1F741
:1044900000002111F5CF2091E80025FF1DC0EC019F
:1044A00080912B01811105C040E050E068E070E090
:1044B00003C070E040E050E0CE010E944E248091A5
:1044C000E8008E778093E80080E2FE01A2ECB2E083
:1044D00001900D928A95E1F7DF91CF910895809335
:1044E000BF027093C1026093C002809103048430C4
:1044F00001F582E08093E9008FEF9091E800815010
:1045000095FD06C095ED9A95F1F700008111F5CF64
:104510008091E80085FF0DC040E050E063E070E06E
:104520008FEB92E00E944E248091E8008E7780937A
:10453000E8000895BC0184E00C946F22BC0183E084
:104540000C946F2280910204811109C00E94DF2522
:104550000E943C268091E20084608093E2000895EE
:104560001092020408950C9416216091FF0381E0DB
:10457000611101C080E00C9401219091030481E05D
:10458000943009F080E06091FF030C94062142E032
:1045900061EC81E00E94582542E261EC82E00E94D9
:1045A00058259091030481E0943009F080E06091F7
:1045B000FF030C940F2180910504833009F461C03E
:1045C00030F4813071F0823009F49AC008958A3055
:1045D00009F486C08B3009F46CC0893009F0A8C09A
:1045E00020C080910404813A09F0A2C08091E800C3
:1045F000877F8093E8008091080490910904892BBB
:1046000021F460E282EC92E003C060E080E090E0A0
:1046100070E00E9499248091E8008B778093E800F5
:10462000089580910404813209F082C080910804C9
:1046300090910904029708F07BC08091E800877F81
:104640008093E8008091E80082FD05C0809103041A
:104650008111F8CF6DC02091F3008091F20090E0BD
:10466000922B029731F48091F100813011F0863065
:1046700021F48091F1008093E2028091E8008B7731
:1046800053C080910404813A09F052C0809108041B
:1046900090910904892B09F04BC08091E800877F35
:1046A0008093E8008091E80080FFFCCF80912B018F
:1046B00036C0809104048132D9F58091080490912C
:1046C0000904892BA9F58091E800877F8093E80091
:1046D0000E948D258091060480932B010C9426085E
:1046E00080910404813221F58091E800877F8093D6
:1046F000E8000E948D25809107048093E3020895CD
:1047000080910404813AA1F48091E800877F80932E
:10471000E8008091E80080FFFCCF8091E302809365
:10472000F1008091E8008E778093E8000C948D254D
:10473000089584B7877F84BF0FB6F894A8958091B9
:104740006000886180936000109260000FBE90E06E
:1047500080E80FB6F89480936100909361000FBEDB
:104760000C9411210E94DF250E943C26E2EEF0E02D
:1047700080818460808378940C94D1288FE191E0CB
:104780000C94DB1F809103048530A9F4809103040D
:10479000853079F40E946221809101048823B1F36D
:1047A0000E942321882391F30E9438240E94260826
:1047B000EDCF0C948D21089508950C94DF23292FBB
:1047C000332723303105C9F060F42130310581F001
:1047D0002230310509F044C08BE390E025E534E058
:1047E00043C021323105E1F02232310549F138C0B0
:1047F00082E190E020E934E037C0992781309105CB
:1048000049F028F0029761F5EBE1F4E005C0E1E53D
:10481000F4E002C0E1E4F4E0849190E09F0124C060
:104820006115710541F061307105D1F489E090E0C6
:1048300020E834E019C089E090E027E634E014C0B5
:104840006115710541F06130710551F486EB90E01E
:1048500022EA34E009C080E490E028E535E004C0B5
:1048600080E090E020E030E0FA0131832083089579
:1048700080E189BD82E189BD09B400FEFDCF809150
:10488000D8008F7D8093D8008091E0008260809373
:10489000E0008091E00081FDFCCF0895CF92DF928F
:1048A000EF92FF920F931F93CF93DF93EC018B0155
:1048B0007A010E94AC25811133C0E114F10439F072
:1048C000F70180819181081B190BC80FD91FC12CDA
:1048D000D12C0115110519F18091E80085FD16C054
:1048E0008091E8008E778093E800E114F10449F0AC
:1048F000F70180819181C80ED91ED182C08285E0E6
:104900000FC00E94AC25882321F30AC089918093AF
:10491000F10001501109FFEFCF1ADF0ADACF80E072
:10492000DF91CF911F910F91FF90EF90DF90CF908B
:10493000089520910A0430910B042617370748F098
:104940006115710539F42091E8002E772093E80075
:1049500001C0B901FC0120E06115710579F1809178
:1049600003048823F1F18530F1F18091E80083FDA3
:104970003CC08091E80082FD2EC08091E80080FF5D
:10498000EBCF2091F3008091F20090E0922B611523
:10499000710551F08830910538F421912093F10090
:1049A000615071090196F3CF21E0089709F020E0EA
:1049B0008091E8008E778093E800CECF2111CFCF91
:1049C0000AC080910304882361F0853061F08091F2
:1049D000E80083FD0AC08091E80082FFF2CF80E00A
:1049E000089582E0089583E0089581E0089520917C
:1049F0000A0430910B042617370748F0611571053A
:104A000039F42091E8002E772093E80001C0B90125
:104A1000FC0120E06115710591F180910304882368
:104A200009F440C0853009F43FC08091E80083FD5F
:104A30003DC08091E80082FD2FC08091E80080FF9A
:104A4000E9CF2091F3008091F20090E0922B611564
:104A5000710559F08830910540F424912093F100BC
:104A60003196615071090196F2CF21E0089709F063
:104A700020E08091E8008E778093E800CBCF211171
:104A8000CCCF0AC080910304882361F0853061F0A7
:104A90008091E80083FD0AC08091E80082FFF2CF98
:104AA00080E0089582E0089583E0089581E008950C
:104AB000982F973068F59093E900981739F0709126
:104AC000EC002091ED005091F00003C0242F762FD0
:104AD00050E021FD02C09F5FECCF3091EB003E7FA4
:104AE0003093EB003091ED003D7F3093ED0030913D
:104AF000EB0031603093EB007093EC002093ED00FD
:104B00005093F0002091EE0027FDE5CF80E008955E
:104B10008F708093E90081E008958091040487FFFD
:104B200011C08091E80082FD05C0809103048111CD
:104B3000F8CF11C08091E8008B770BC080910304FF
:104B4000882349F08091E80080FFF8CF8091E80049
:104B50008E778093E80008952091E4003091E5007D
:104B600095E64091EC00842F817040FF23C0809136
:104B7000E80080FD1DC080910304882399F08530F2
:104B800099F08091EB0085FD11C04091E4005091B7
:104B9000E5002417350729F3915011F09A01E1CF70
:104BA00084E0089582E0089583E0089581E0089507
:104BB00080E008954091E80042FFDDCF08950E9413
:104BC0004D260E945526E0EEF0E0808181608083D2
:104BD000E8EDF0E080818F77808319BCA7EDB0E02D
:104BE0008C918E7F8C9380818F7E808310920204C3
:104BF00008950F931F93CF93DF930E944D260E9439
:104C00005526C8EDD0E088818F77888388818068B9
:104C1000888388818F7D888319BC10920304109249
:104C2000FF03109201041092000400EE10E0F8015E
:104C300080818B7F808388818160888342E060E00F
:104C400080E00E945825E1EEF0E080818E7F808335
:104C5000E2EEF0E0808181608083808188608083E3
:104C6000F80180818E7F8083888180618883DF91D5
:104C7000CF911F910F910895E8EDF0E080818F7E34
:104C80008083E7EDF0E080818160808384E082BFF3
:104C900081E0809302040C94F925E8EDF0E0808136
:104CA0008E7F80831092E20008951092DA001092B5
:104CB000E10008951F920F920FB60F9211242F93C7
:104CC0003F934F935F936F937F938F939F93AF9394
:104CD000BF93EF93FF938091E10082FF0BC080911F
:104CE000E20082FF07C08091E1008B7F8093E100AA
:104CF0000E94D0288091DA0080FF1FC08091D800E8
:104D000080FF1BC08091DA008E7F8093DA00809153
:104D1000D90080FF0DC080E189BD82E189BD09B461
:104D200000FEFDCF81E0809303040E94A22205C013
:104D300019BC109203040E94B0228091E10080FF10
:104D400019C08091E20080FF15C08091E2008E7F43
:104D50008093E2008091E20080618093E200809184
:104D6000D80080628093D80019BC85E0809303044A
:104D70000E94B5228091E10084FF30C08091E20062
:104D800084FF2CC080E189BD82E189BD09B400FEA9
:104D9000FDCF8091D8008F7D8093D8008091E10075
:104DA0008F7E8093E1008091E2008F7E8093E2000D
:104DB0008091E20081608093E2008091FF0388236C
:104DC00011F084E007C08091E30087FD02C081E01C
:104DD00001C083E0809303040E94BD228091E10022
:104DE00083FF29C08091E20083FF25C08091E1000C
:104DF000877F8093E10082E0809303041092FF0399
:104E00008091E1008E7F8093E1008091E2008E7FAF
:104E10008093E2008091E20080618093E20042E0B2
:104E200060E080E00E9458258091F00088608093C7
:104E3000F0000E94B322FF91EF91BF91AF919F913B
:104E40008F917F916F915F914F913F912F910F9033
:104E50000FBE0F901F9018951F920F920FB60F92D2
:104E600011242F933F934F935F936F937F938F936F
:104E70009F93AF93BF93CF93DF93EF93FF93C09133
:104E8000E900CF708091EC00D82FD17080FDD0E880
:104E90001092E9008091F000877F8093F000789471
:104EA0000E9470271092E9008091F0008860809342
:104EB000F000CD2BCF70C093E900FF91EF91DF910F
:104EC000CF91BF91AF919F918F917F916F915F91A2
:104ED0004F913F912F910F900FBE0F901F901895FB
:104EE0001F93CF93DF93CDB7DEB7AA970FB6F89491
:104EF000DEBF0FBECDBFE4E0F4E08091F10081930E
:104F000024E0EC30F207C9F70E94DB228091E80030
:104F100083FF2EC18091040490910504492F50E035
:104F20004A30510508F024C1FA01EE59FF4F0C94A4
:104F30004429803821F0823809F01AC108C08091D4
:104F4000000490910104992389F082600FC0809140
:104F500008048F70873008F00BC18093E9008091BE
:104F6000EB0085FB882780F91092E9009091E8001A
:104F7000977F9093E8008093F1001092F100D1C0E8
:104F8000282F2D7F09F0F4C0882319F0823061F0BA
:104F9000EFC080910604813009F0EAC0933009F037
:104FA00080E0809301042EC08091060481112AC004
:104FB000809108048F702FEF280F263008F0D8C09A
:104FC0008093E9002091EB0020FF1CC0933021F476
:104FD0008091EB00806214C09091EB0090619093FF
:104FE000EB0021E030E0A90102C0440F551F8A9573
:104FF000E2F74093EA001092EA008091EB008860AB
:105000008093EB001092E9008091E800877F809305
:10501000E8000E948D25ACC08111AAC01091060441
:105020001F778091E3008078812B8093E30080914B
:10503000E800877F8093E8000E948D258091E8003A
:1050400080FFFCCF8091E30080688093E300111122
:1050500002C082E001C083E08093030489C08058CD
:10506000823008F085C080910604909107048C3D41
:1050700053E0950779F583E08A838AE289834FB705
:10508000F894DE01139620E03EE051E2E32FF0E0D9
:1050900050935700E49120FF03C0E295EF703F5F0B
:1050A000EF708E2F90E0EA3010F0C79601C0C096E6
:1050B0008D939D932F5F243149F74FBF8091E80076
:1050C000877F8093E8006AE270E0CE0101960E943B
:1050D000992416C06091080470910904AE014F5FD5
:1050E0005F4F0E94DD23BC01892B09F441C09091E0
:1050F000E800977F9093E80089819A810E94F724C5
:105100008091E8008B778093E80032C0803881F589
:105110008091E800877F8093E8008091FF0380936F
:10512000F1008091E8008E7772CF811121C08091CB
:1051300006049091070499270297D4F48091E8001F
:10514000877F8093E800809106048093FF030E948C
:105150008D258091FF03811106C08091E30087FDBA
:1051600002C081E001C084E0809303040E94C72252
:105170008091E80083FF0AC08091E800877F8093D8
:10518000E8008091EB0080628093EB00AA960FB656
:10519000F894DEBF0FBECDBFDF91CF911F91089570
:1051A0000895CF93809103048823A1F0C091E90072
:1051B000CF709091EC00892F817090FD80E8C82B12
:1051C0001092E9008091E80083FD0E947027CF7063
:1051D000C093E900CF91089587FB082E062687FD2E
:1051E000819567FD61950E947B290EF4919507FCDE
:1051F00081950895AA1BBB1B51E107C0AA1FBB1FC5
:10520000A617B70710F0A61BB70B881F991F5A9552
:10521000A9F780959095BC01CD01089597FB072EC5
:1052200016F4009407D077FD09D00E94FA2807FCF5
:1052300005D03EF4909581959F4F089570956195A6
:105240007F4F0895A1E21A2EAA1BBB1BFD010DC0C2
:10525000AA1FBB1FEE1FFF1FA217B307E407F50726
:1052600020F0A21BB30BE40BF50B661F771F881F02
:10527000991F1A9469F760957095809590959B0198
:10528000AC01BD01CF010895EE0FFF1F0590F49111
:10529000E02D09940E945229332312F48A1B9B0BA0
:1052A0000C946329A29FB001B39FC001A39F700D0E
:1052B000811D1124911DB29F700D811D1124911D1E
:1052C00008950E945229B7FF0895821B930B0895F9
:1052D0000E945229A59F900DB49F900DA49F800D10
:1052E000911D11240895B7FF0C9468290E94682924
:1052F000821B930B0895991B79E004C0991F9617A0
:1053000008F0961B881F7A95C9F780950895FC01CF
:105310004150504030F001900616D1F73197CF013F
:105320000895882799270895FB01DC0104C08D9119
:105330000190801921F441505040C8F7881B990B07
:105340000895F999FECF92BD81BDF89A992780B54D
:105350000895A6E1B0E044E050E00C94DB29A8E118
:10536000B0E042E050E00C94DB29262FF999FECF03
:1053700092BD81BDF89A019700B4021639F01FBAA8
:1053800020BD0FB6F894FA9AF99A0FBE08950396C5
:10539000272F0E94B6290E94B529252F0E94B629E1
:1053A000242F0C94B6290196272F0E94B6290C941D
:1053B000B529DC01CB01FC01F999FECF06C0F2BD95
:1053C000E1BDF89A319600B40D9241505040B8F7C3
:0653D0000895F894FFCFE0
:1053D600C8006002280850011E0A140101010200DB
:1053E6005400545401191A1B1C1D1E1F2021220B88
:1053F600222E220F229E229A220E2201E200E9008C
:10540600EA00B500B600B700CD008301CC008A01E2
:105416009201940121022302240225022602270278
:105426002A02B300B4006F007000818283E200E9B3
:1054360000EA00B500B600B700CD008301CC008AB3
:105446000192019401210223022402250226022749
:10545600022A02B300B4006F007000818283F0F16B
:10546600C66766369431373534979633F490919201
:1054760093950001020202020606060909090909B6
:10548600090F0F0F0F0F0F151515181919191919DF
:0854960019191919192324004A
:00000001FF
